:020000040800F2
:10000000000001208D3300084D3100084F310008F9
:10001000513100085331000855310008000000003C
:100020000000000000000000000000005731000840
:1000300059310008000000005B3100085D31000804
:10004000D5330008D5330008D5330008D533000870
:10005000D5330008D5330008D5330008D533000860
:10006000D5330008D5330008D5330008D533000850
:10007000D5330008D5330008613100086D31000820
:100080007931000885310008D5330008D5330008E0
:10009000D5330008D5330008D5330008D533000820
:1000A000D5330008D5330008D5330008D533000810
:1000B000D5330008D5330008D5330008D533000800
:1000C000D5330008D5330008D5330008D5330008F0
:1000D000D5330008913100089D310008D533000860
:1000E000D5330008D5330008D5330008D5330008D0
:1000F000D5330008D5330008D5330008D5330008C0
:10010000D5330008D5330008D5330008D5330008AF
:10011000D5330008D5330008A9310008D5330008CD
:10012000D5330008D5330008D5330008D53300088F
:1001300000000000000000000000000000000000BF
:1001400000000000000000000000000000000000AF
:10015000000000000000000000000000000000009F
:10016000000000000000000000000000000000008F
:10017000000000000000000000000000000000007F
:10018000000000000000000000000000000000006F
:10019000000000000000000000000000000000005F
:1001A000000000000000000000000000000000004F
:1001B000000000000000000000000000000000003F
:1001C000000000000000000000000000000000002F
:1001D000000000000000000000000000000000001F
:0401E0005FF8E0F1F3
:1001E40010B5054C237833B9044B13B10448AFF36D
:1001F40000800123237010BD800200200000000055
:100204008844000808B5034B1BB103490348AFF306
:10021400008008BD0000000084020020884400081B
:10022400D0400B1CD1409C46203AD3401843524244
:10023400634693401843704738B50E4B054618780B
:100244004FF47A73B3FBF0F30B4A1068B0FBF3F08E
:1002540000F09EF8044658B90F2D09D802462946E5
:100264004FF0FF3000F054F8044B20461D6038BDB9
:10027400012038BD000000201402002004000020EA
:10028400074A08B51368032043F01003136000F015
:100294002DF80020FFF7D0FF02F038FE002008BD43
:1002A40000200240034A044B11681B780B4413607E
:1002B400704700BF0403002000000020014B1868B1
:1002C400704700BF0403002038B50446FFF7F6FF6B
:1002D4000546631C1EBF044B1B78E418FFF7EEFFB2
:1002E400401B8442FAD838BD00000020074A0002AF
:1002F400D36800F4E06023F4E0631B041B0C43F0B8
:10030400BF6343F400330343D360704700ED00E060
:10031400174B30B5DC68C4F30224C4F10703251D70
:10032400042B28BF0423062D4FF0010598BF002499
:1003340005FA03F303F1FF3388BF033C1940A140DE
:1003440005FA04F4013C2240002842EA01024FEA83
:100354000212AFBF00F16040064B00F00F00D2B2B2
:10036400A5BFD2B200F561401A5480F8002330BD15
:1003740000ED00E014ED00E00123420900F01F004D
:1003840003FA00F0014B43F82200704700E100E05B
:100394000138B0F1807F0AD2F021064B064A58603A
:1003A40082F823100020072298601A607047012009
:1003B400704700BF10E000E000ED00E010B5002839
:1003C40032D00168194B1424994225D8184AA3F253
:1003D40007430A44B2FBF4F2920002648468C363E4
:1003E40043680A682343C46822F47F5223430469A0
:1003F40022F0300223434469234384692343C469BC
:10040400234313430B600122002380F821208363DC
:1004140080F82030184610BD064B0B44B3FBF4F3B0
:100424009B000364044BD9E7012010BD070402407C
:10043400F8FFFDBFF8FBFDBF00040240F0B590F8E3
:100444002040012C35D0012490F8215080F8204020
:10045400A5424FF000064FF0020428D180F8214055
:10046400046886632668076C26F001062660C66B5E
:10047400BD407560636043680568102BC36A0BBF99
:10048400A260A160E160E2604BB1236843F00E0317
:1004940023602B68002043F001032B60F0BD236828
:1004A40023F004032360236843F00A03F0E780F891
:1004B40020600220F0BD000090F8213010B5022B1E
:1004C40003D004238363012010BD03681A6822F05B
:1004D4000E021A601A6822F001021A60294A934235
:1004E40024D902F56272934219D01432934218D07F
:1004F4001432934217D0143293420CBF4FF48053FA
:100504004FF48033204A53600123002480F82130C3
:10051400436B80F820409BB39847204610BD0123CD
:10052400F0E71023EEE74FF48073EBE717498B42B3
:1005340016D014318B4215D014318B4214D014319F
:100544008B4214D014318B4214D014318B4214D00A
:10055400934214BF4FF480334FF080730C4AD2E7B8
:100564000123FBE71023F9E74FF48073F6E74FF418
:100574008053F3E74FF48033F0E74FF48013EDE753
:10058400184610BD800002400004024008000240EA
:100594000000024070B40425C66B026C3468036822
:1005A40095402542196855D04D0753D51A689606CB
:1005B4005EBF1A6822F004021A60604A93421FD98F
:1005C40002F56272934214D01432934213D014325F
:1005D400934212D0143293420CBF4FF480434FF431
:1005E4008023574A5360C36A002B00F0A58070BC77
:1005F40018470423F5E74023F3E74FF48063F0E75B
:1006040050498B4216D014318B4215D014318B4291
:1006140014D014318B4214D014318B4214D01431C1
:100624008B4214D0934214BF4FF480234FF0806365
:10063400454AD7E70423FBE74023F9E74FF48063F7
:10064400F6E74FF48043F3E74FF48023F0E74FF4E9
:100654008003EDE702259540254257D08D0755D5F7
:100664001A68940606D41A6822F00A021A60012253
:1006740080F82120314A93421ED902F562729342D6
:1006840013D01432934212D01432934211D0143244
:1006940093420CBF4FF400534FF40033284A536085
:1006A400002380F82030836A9EE70223F6E72023A4
:1006B400F4E74FF40073F1E722498B4216D014316A
:1006C4008B4215D014318B4214D014318B4214D088
:1006D40014318B4214D014318B4214D0934214BF82
:1006E4004FF400334FF00073174AD8E70223FBE7B7
:1006F4002023F9E74FF40073F6E74FF40053F3E7D0
:100704004FF40033F0E74FF40013EDE7082595406C
:10071400254211D009070FD5196821F00E0119607F
:10072400012303FA02F27260836380F8213000230C
:1007340080F82030036B57E770BC7047800002409C
:10074400000402400800024000000240114AD3683D
:1007540013F0100305D01049CB6943F00203CB61B9
:100764001023D268500706D50B4943F00403CA6925
:1007740042F00102CA61074AD169C90708D506488F
:10078400C16941F00401C161D16921F00101D16164
:10079400D36070470020024008030020064B18690C
:1007A40010F0800007D0054A5A6002F188325A607E
:1007B4001869C0F3C0107047002002402301674548
:1007C400034A0020136943F080031361704700BF9C
:1007D40000200240F8B50646FFF770FD114C0746AD
:1007E4002546E368D80712D4E368990644BF20235A
:1007F400E360EB68DA0606D4EB69DB0703D4E86848
:1008040010F0040002D0FFF7A1FF0120F8BD731C13
:10081400E7D00EB90320F8BDFFF750FDC01B864298
:10082400DFD2F7E7002002402DE9F84F1F4C99462C
:10083400237E0546012B0F46904633D001234CF20C
:1008440050302376FFF7C6FF40BB012D03D0022DA5
:100854000CBF022504250026B246DFF854B032014D
:1008640040464946FFF7DCFCC4F81CA0DBF8103016
:1008740080B243F00103CBF8103027F816004CF295
:100884005030FFF7A7FFDBF8103023F00103CBF85B
:10089400103018B90136F3B29D42E0D80023237614
:1008A400BDE8F88F0220BDE8F88F00BF08030020E0
:1008B400002002400022064BDA61064B1A6942F01E
:1008C40004021A611A6942F040021A61704700BFBB
:1008D40008030020002002400022064BDA61064B88
:1008E4001A6942F002021A6158611A6942F0400220
:1008F4001A61704708030020002002402DE9F041EE
:10090400234D07462B7E8846012B3DD001240368E6
:100914002C76022B4CF2503013D1FFF75BFF20B141
:10092400012000232B76BDE8F081FFF7C3FF4CF2D2
:100934005030FFF74FFF174A136923F00403136184
:10094400EFE7FFF747FF0028EAD14FF0FF33C8F87D
:1009540000302046BE680F4CFA68BB6803EBC22324
:100964009E42DED23046FFF7B7FF4CF25030FFF71D
:1009740031FF236923F00203236110B1C8F800603A
:10098400CFE706F50066E7E70220BDE8F08100BF87
:1009940008030020002002402DE9F74F00221646EC
:1009A4006C4F6D4BDFF8B8E1DFF8B8C14FF00108C8
:1009B4000C6808FA06F808EA0404A04540F08580AB
:1009C4004D68122D00F0B78000F28D80022D00F0EA
:1009D400AF8000F28180002D00F09180012D00F0A5
:1009E400A5804FF00F09FF2C93BF824606F1804586
:1009F400083DD0F800B092BFB500D0F804B0AD0007
:100A040009FA05F82BEA080802FA05F588BF00F18F
:100A1400040A48EA0505CAF80050D1F804A01AF0FF
:100A2400805F52D0BD6926F0030845F00105BD6121
:100A3400BD6908F1804805F00105019508F5803885
:100A440006F0030B019D4FEA8B0BD8F8085009FA06
:100A54000BF925EA0909414DA84271D005F58065D5
:100A6400A8426FD005F58065A8426DD005F5806574
:100A7400A8426BD005F58065A84269D070450CBFCB
:100A84000525062505FA0BF545EA0905C8F80850B9
:100A94001D681AF4803F14BF2543A5431D605D689B
:100AA4001AF4003F14BF2543A5435D609D681AF402
:100AB400801F14BF2543A5439D60DD681AF4001F01
:100AC40014BF2C4325EA0404DC600136102E7FF4A5
:100AD4006DAF03B0BDE8F08F032D25D0112D80D16B
:100AE400CA6804327DE7654509D012D8DFF87890EA
:100AF4004D4504D009F580394D457FF472AF8A68BD
:100B0400E2B1012A0CBFC0F81080C0F8148008229A
:100B140067E7DFF858904D45F1D009F580394D4528
:100B2400EDD0A9F58019E7E700225AE7CA6858E72B
:100B3400CA68083255E7CA680C3252E7042250E703
:100B440000259FE701259DE702259BE7032599E7FB
:100B5400042597E70010024000040140000801400A
:100B6400001C014000002110000011100000311091
:100B74000AB1016170470904FBE70268536913F481
:100B840080630DD06FF480635361042320220364D7
:100B94000023036380F83C3080F83D200120704737
:100BA400184670472DE9F843044617469946C1F3A1
:100BB40007488EB22568B8F1010F0CBF6B69AB69A9
:100BC40036EA030314BF0120002008B9BDE8F88306
:100BD4006B695A0512D52B68202243F400732B60ED
:100BE4006FF480636B610423236400230120236377
:100BF40084F83C3084F83D20BDE8F8837B1CD9D0D0
:100C04004FB900232022236384F83C3084F83D202C
:100C14000320BDE8F883FFF751FBA0EB09008742EE
:100C2400C8D2EEE72DE9F843044690461F46089ED5
:100C3400C1F307498DB22368B9F1010F0CBF5B6999
:100C44009B6935EA03030CBF01230023434502D00B
:100C54000020BDE8F8837B1CEDD05FB9002320227F
:100C6400236384F83C3084F83D20032084F83E302C
:100C7400BDE8F883FFF722FB801B8742DBD2EDE758
:100C840070B504460D46164623685B691B0601D5FC
:100C9400002070BD2046FFF770FFA8B96A1CF3D08E
:100CA40065B9236C202243F020032364002303202E
:100CB400236384F83C3084F83D2070BDFFF7FEFACE
:100CC400801B8542E0D2ECE7012070BD2DE9FF4195
:100CD40015460268984613680B9E43F480731360AC
:100CE4000F4600960A9B00224FF001110446FFF7BD
:100CF40099FF68B9236807F0FE071F610A9A334613
:100D04001A492046FFF74EFF30B1236C042B18D04C
:100D1400032004B0BDE8F081236803905A690A995E
:100D240003929B69324603932046039BFFF7A8FF77
:100D340048B1236C042BEBD12268136843F400738D
:100D440013600120E5E7B8F1010F236802D1EDB289
:100D54001D61DEE72A0A1A610A9932462046FFF726
:100D64008FFF0028E5D12368F1E700BF02000100EE
:100D74002DE9FF419846036816461A680B9D42F414
:100D840080621A601A680F4642F480721A604FF04B
:100D9400011100950A9B00220446FFF743FF80B926
:100DA4002368FFB207F0FE021A612D492B460A9A06
:100DB4002046FFF7F7FE40B1236C042B01D101203C
:100DC40000E0032004B0BDE8F081236803905A6971
:100DD4000A9903929B692A4603932046039BFFF7D3
:100DE4004FFF40B1236C042BEBD12268136843F40A
:100DF40000731360E3E7B8F1010F236824D1F6B25E
:100E04001E612A460A992046FFF73AFF0246002847
:100E1400E8D1216820460B6843F480730B60009589
:100E24000A9B4FF00111FFF7FDFE0028C9D123688A
:100E340047F001071F610A9A2B4609492046FFF72C
:100E4400B1FE0028B8D1BDE7320A1A610A992A46D0
:100E54002046FFF715FF0028C4D12368CFE700BF61
:100E64000200010070B504460D4616462068436929
:100E740013F0400301D0002070BD4269D2060BD5A7
:100E84006FF0100242612022236484F83C30236313
:100E9400012084F83D2070BD5DB9236C032043F02C
:100EA40020032364202384F83D30002384F83C305D
:100EB40070BDFFF703FA801B8542D7D2EDE770B50A
:100EC40004460D46164623685B695B0701D500207E
:100ED40070BD2046FFF751FEA8B96A1CF3D065B96E
:100EE400236C202243F02003236400230320236384
:100EF40084F83C3084F83D2070BDFFF7DFF9801B97
:100F04008542E0D2ECE7012070BD000038B504460C
:100F140008B9012038BD90F83D3003F0FF021BB939
:100F240080F83C2002F014F82423226884F83D3031
:100F3400136823F00103136000F098FC63682F4AE0
:100F4400934230D82E4A9042E3D92E4A2168B0FB0E
:100F5400F2F24A6001320A62284A0138934232D8D6
:100F64005B00B0FBF3F0431CC3F30B03042B38BF4B
:100F74000423CB61226AE369002013430B60E26817
:100F8400236913438B60A26963691343CB600B68C5
:100F940043F001030B602023206484F83D30206378
:100FA40084F83E0038BD184A9042B2D9154D4FF42A
:100FB4009672B0FBF5F521686A434D604FF47A757B
:100FC400B2FBF5F2C6E7A26852B903EB4303B0FBE8
:100FD400F3F0431CC3F30B036BB143F40043C8E7C2
:100FE40019225343B0FBF3F0431CC3F30B0313B1B7
:100FF40043F44043BDE70123BBE700BFA0860100E3
:101004007F841E0040420F00FF083D002DE9F34796
:1010140004469A46884691460C9EFFF74FF994F889
:101024003D300546202B03D0022002B0BDE8F087F6
:101034000090192301223E492046FFF7F3FD0028C2
:10104400F2D194F83C30012BEED0012384F83C30EB
:10105400236800271A684146D20758BF1A682046F9
:101064005CBF42F001021A601A6822F400621A603E
:10107400212384F83D30402384F83E300A9B2764C2
:101084006362BDF82C30019563852A4B0096E362B8
:10109400638D4A4623855346FFF718FE00282AD05D
:1010A400236C84F83C70042B07D10120BDE7FFF7C3
:1010B400E7FD20B1236C042B34D00320B5E7616A2B
:1010C40027684B1C63620B78228D3B61638D501E35
:1010D400013B9BB263857B6980B25B0720850AD59F
:1010E40048B18B1C63624B78023A3B61638D228565
:1010F400013B9BB26385238D2A4631462046002B53
:10110400D5D1FFF7DCFE0028D4D12268136843F45C
:1011140000731360202384F83C0084F83D3084F885
:101124003E0082E72268136843F400731360BCE74F
:10113400020010000000FFFF2DE9F047044686B0CE
:101144009A460D469146109FFFF7B8F894F83D3043
:101154000646202B04D00225284606B0BDE8F087B9
:1011640000901923012281492046FFF75BFD0028E6
:10117400F1D194F83C30012BEDD0012384F83C30BC
:1011840023684FF000081A682946D20758BF1A6826
:1011940020465CBF42F001021A601A6822F4006221
:1011A4001A60222384F83D30402384F83E300E9B9D
:1011B400C4F840806362BDF83C30019663856C4B93
:1011C4000097E362638D4A4623855346FFF7D0FDBB
:1011D400054630B1236C84F83C80042B3DD10125B5
:1011E400BAE7228D236892B902905A6902929A69E9
:1011F4000292029A1A6842F400721A60202384F858
:101204003D30002384F83E3084F83C30A4E7012AC2
:1012140025D11A6822F480621A6072B6236803909A
:101224005A6903929A690392039A1A6842F4007203
:101234001A6062B6DFF83C81238D002BDED0032BCD
:1012440077D8012B27D1324639462046FFF70AFECC
:1012540000283FD0236C202BC1D103257CE7022A30
:101264001A680ED142F400621A6072B623680490C0
:101274005A6904929A690492049A1A6822F4806260
:10128400D6E742F480621A6005905A6905929B6918
:101294000593059BCEE7022B00963B464FF00002D8
:1012A4004146204624D1FFF7BDFC0028D5D172B6B3
:1012B40023681A6842F400721A60626A1B69511C3E
:1012C40061621370238D013B2385638D013B9BB2C7
:1012D400638562B6636A5A1C6262226812691A7074
:1012E400238D013B2385638D013B9BB26385A3E77B
:1012F400FFF798FC02460028AFD121680B6823F45D
:1013040080630B6072B6636A2046591C616221686F
:1013140009691970238D0096013B2385638D41462D
:10132400013B9BB263853B46FFF77CFC0028BFD0A2
:1013340093E7324639462046FFF794FD002889D1C9
:10134400636A5A1C6262226812691A70238D2268C9
:10135400013B2385638D013B9BB2638553695B0726
:101364007FF56AAF636A591C6162B7E70200100037
:101374000000FFFF0400010003682DE9F341DB07CF
:10138400054610D42B689F075ED42B68190700F11B
:1013940095802B685A0700F1BF80EA69002A40F063
:1013A4002D81002014E0904C636803F00C03042B9F
:1013B40007D0636803F00C03082B0CD16368DE03C9
:1013C40009D523689C03DDD56B68002BDAD1012095
:1013D40002B0BDE8F0816B68B3F5803F10D123689B
:1013E40043F480332360FEF769FF064623689803BD
:1013F400C8D4FEF763FF801B6428F7D90320E7E70E
:101404009BB9236823F480332360236823F4802367
:101414002360FEF753FF064623689903B2D5FEF70F
:101424004DFF801B6428F7D9E8E7B3F5A02F2368A4
:1014340003D143F480232360D1E723F48033236072
:10144400236823F48023CDE7674C636813F00C0F03
:1014540007D0636803F00C03082B10D16368DA0328
:101464000DD423689B0702D52B69012BAFD12368C8
:101474006A6923F0F80343EAC203236085E72A6913
:101484005A4B6AB101221A60FEF718FF0646236818
:101494009F07ECD4FEF712FF801B0228F7D9ADE7B3
:1014A4001A60FEF70BFF0646236898077FF56DAFB9
:1014B400FEF704FF801B0228F6D99FE7AA694A4C6D
:1014C4004B4BDAB101221A60FEF7F8FE0646636A56
:1014D4009B070DD54FF4FA52464B1B68B3FBF2F34E
:1014E400019300BF019B5A1E0192002BF9D150E7D2
:1014F400FEF7E4FE801B0228E9D97FE71A60FEF7B5
:10150400DDFE0646636A9F077FF543AFFEF7D6FE0E
:10151400801B0228F6D971E7334CE369D80024D440
:101524000127E36943F08053E361E36903F08053E7
:101534000093009B304E3368D90518D5EB68012B16
:1015440026D1236A43F001032362FEF7B7FE41F27A
:1015540088368046236A9B073FD5002F3FF41DAF92
:10156400E36923F08053E36117E70027E2E7336878
:1015740043F480733360FEF7A1FE80463368DA05D6
:10158400DCD4FEF79BFEA0EB08006428F6D935E70F
:10159400ABB9236A41F2883823F001032362236A3A
:1015A40023F004032362FEF789FE0646236A9807A4
:1015B400D3D5FEF783FE801B4045F7D91EE7052BE4
:1015C400236A03D143F004032362BAE723F001033F
:1015D4002362236A23F00403B6E7FEF76FFEA0EB51
:1015E4000800B042B6D909E70010024000004242A8
:1015F400800442421402002000700040224C6368C0
:1016040003F00C03082B3FF4E2AE00231F4E022A22
:1016140033602BD1FEF752FE0746236899011FD48D
:101624002B6AB3F5803F05D16268A96822F40032C1
:101634000A436260696A62680B4322F474121343BA
:10164400636001233360FEF739FE054623689A017F
:101654003FF5A7AEFEF732FE401B0228F6D9CDE6D1
:10166400FEF72CFEC01B0228D7D9C7E6FEF726FEDC
:10167400054623689B017FF594AEFEF71FFE401BD1
:101684000228F6D9BAE600BF0010024060004242C8
:1016940030B5194B87B002AC03F110052246186827
:1016A4005968083303C2AB421446F7D101238DF8BD
:1016B4000430022311498DF805304B6803F00C0205
:1016C400082A17D1C3F3834206A80244DB0312F8A5
:1016D400102C0CD54B680A48C3F34043504306AA68
:1016E400134413F8143CB0FBF3F007B030BD0548C5
:1016F4005043FAE70248F8E7A0440008001002400B
:1017040000127A0000093D00544A2DE9F0411368A3
:10171400054603F007038B420E462AD329688C073B
:1017240034D4CA0747D44D4A136803F007039E42D2
:10173400C0F082802A684A4C12F0040F40F087807F
:10174400130706D563682A6923F4605343EAC20386
:101754006360FFF79DFF6368424AC3F30313D35CDE
:10176400D840414B18600020FEF766FD0020BDE81C
:10177400F081136823F007030B431360136803F02D
:1017840007039942CAD00120BDE8F081344B11F01F
:10179400040F1EBF5A6842F4E0625A60080742BF51
:1017A4005A6842F460525A605A68A86822F0F002FB
:1017B40002435A60B5E76A68294C012A23681CD1A0
:1017C40013F4003FDFD0636841F2883823F0030349
:1017D40013436360FEF772FD6B680746012B14D157
:1017E400636803F00C03042B9DD0FEF767FDC01B58
:1017F4004045F5D90320BDE8F081022A02D113F057
:10180400007FDFE713F0020FDCE7022B0FD16368E0
:1018140003F00C03082B86D0FEF750FDC01B404597
:10182400F5D9E7E7FEF74AFDC01B4045E2D86368F7
:1018340013F00C0FF6D176E7136823F00703334354
:101844001360136803F007039E429CD172E7636838
:10185400E96823F4E0630B43636071E7002002400E
:10186400001002402D4C000814020020044B054ACD
:101874005B68C3F30223D35C034A1068D840704703
:10188400001002403D4C000814020020044B054A9D
:101894005B68C3F3C223D35C034A1068D840704723
:1018A400001002403D4C0008140200200368002090
:1018B400DA6842F00102DA601A6842F001021A6042
:1018C40070477047704770477047036810B51A69CE
:1018D400044691070ED5DA6892070BD56FF0020221
:1018E4001A6101229B6902779B0777D0FFF7EAFF11
:1018F4000023237723681A69500710D5DA68510743
:101904000DD56FF004021A6102229B69227713F449
:10191400407F204668D0FFF7D5FF00232377236854
:101924001A6912070FD5DA6810070CD56FF0080290
:101934001A610422DB692277990720465AD0FFF7FF
:10194400C1FF0023237723681A69D20610D5DA6809
:10195400D0060DD56FF010021A610822DB692277D8
:1019640013F4407F20464BD0FFF7ACFF00232377CE
:1019740023681A69D10708D5DA68D20705D56FF04C
:10198400010220461A6101F087F923681A691006DA
:1019940008D5DA68110605D56FF0800220461A6171
:1019A40000F0BFF823681A69520608D5DA685006B1
:1019B40005D56FF0400220461A61FFF785FF2368C2
:1019C4001A69910622D5DA6892061FD56FF02002B3
:1019D4002046BDE810401A6100F0A2B8FFF771FF7D
:1019E4002046FFF770FF83E7FFF76BFF2046FFF702
:1019F4006AFF92E7FFF765FF2046FFF764FFA0E761
:101A0400FFF75FFF2046FFF75EFFAFE710BD000062
:101A1400244A0368904212D002F5006290420ED02C
:101A2400B0F1804F0BD0A2F59832904207D002F566
:101A34008062904203D002F5806290421DD14A68D0
:101A440023F070031343174A904212D002F5006248
:101A540090420ED0B0F1804F0BD0A2F59832904254
:101A640007D002F58062904203D002F58062904272
:101A740003D1CA6823F4407313434A6923F08003F3
:101A8400134303608B68C3620B688362054B9842FF
:101A940003D003F50063984201D10B69036301236A
:101AA40043617047002C014010B50446A0B190F882
:101AB4003D3003F0FF021BB980F83C2001F07AFAB4
:101AC4000223206884F83D30211DFFF7A1FF012384
:101AD400002084F83D3010BD012010BD90F83C304A
:101AE40010B5012B4FF0020318D080F83D30036885
:101AF4000C685A68496822F070025A605A68224396
:101B04005A609A6822F080029A609A680A439A603E
:101B1400012380F83D30002380F83C30184610BD86
:101B2400704770470368DA6822F49072DA605A6981
:101B340022F001025A61202380F83A3070470000F5
:101B44002DE9F0470568C2682B69016923F4405305
:101B540013432B618368EA680B43416922F4B05252
:101B640022F00C020B431343EB606B69826923F48C
:101B7400407313436B61404B81469D424FF01904FF
:101B840046D1FFF783FE04FB00F3D9F804604FF05D
:101B94006408B600B3FBF6F3B3FBF8F31E01FFF7DA
:101BA40075FE6043D9F804309B00B0FBF3F7FFF7F0
:101BB4006DFE6043D9F804309B00B0FBF3F3B3FB34
:101BC400F8F308FB13731B013233B3FBF8F303F090
:101BD400F007FFF75BFE6043D9F804209200B0FBE6
:101BE400F2FAFFF753FE6043D9F804309B00B0FBD0
:101BF400F3F3B3FBF8F308FB13A31B013233B3FB7A
:101C0400F8F303F00F033B433344AB60BDE8F087C4
:101C1400FFF72CFE04FB00F3D9F804604FF06408CE
:101C2400B600B3FBF6F3B3FBF8F31E01FFF71EFE99
:101C34006043D9F804309B00B0FBF3F7FFF716FEBE
:101C44006043D9F804309B00B0FBF3F3B3FBF8F323
:101C540008FB13731B013233B3FBF8F303F0F007F3
:101C6400FFF704FE6043D9F804209200B0FBF2FAB7
:101C7400FFF7FCFDB7E700BF00380140F8B50446A4
:101C84000E4617461D4621680B6836EA030301D148
:101C94000020F8BD6B1CF7D095B923680320DA68DF
:101CA40022F4D072DA605A6922F001025A612023C8
:101CB40084F8393084F83A30002384F83830F8BD99
:101CC400FEF7FCFAC01B8542DDD2E6E710B50446F8
:101CD40040B390F8393003F0FF021BB980F8382084
:101CE40001F07CF92423226884F83930D368204633
:101CF40023F40053D360FFF723FF236800201A69FD
:101D040022F490421A615A6922F02A025A61DA686E
:101D140042F40052DA602023E06384F8393084F816
:101D24003A3010BD012010BD2DE9F0411F4690F856
:101D340039300446202B0D4690464ED1002949D017
:101D4400002A47D090F83830012B46D0012380F880
:101D540038300023C363212380F83930FEF7AEFA0C
:101D64000646A4F82480A4F82680E38C9BB26BB9C1
:101D74003B46324640212046FFF780FFA8B9202386
:101D840084F8380084F83930BDE8F081E38C3246B9
:101D9400013B9BB2E384A3688021B3F5805F2046B6
:101DA4003B460ED1FFF76AFF10B10320BDE8F08176
:101DB4002B882268C3F308035360236943B90235AF
:101DC400D3E7FFF75BFF0028EFD123682A785A6036
:101DD4000135CAE70120BDE8F0810220BDE8F081A9
:101DE400134690F83A2073B5202A054638D10029C5
:101DF40034D0002B32D090F83820012A30D0012280
:101E0400002480F83820222281628385C46380F80C
:101E14003A20406B134A2E688262134A4463C262BA
:101E2400124A02630A46311DFEF708FB20462B685E
:101E340001941A6801925A6885F838400192019A0F
:101E4400DA6842F48072DA605A6942F001025A6137
:101E54005A6942F040025A6102B070BD0120FBE7AA
:101E64000220F9E7771E00082D1F0008391F00081B
:101E7400704708B50368426A1B6813F0200310D149
:101E8400D3851368D96821F48071D960596921F028
:101E940001015961596921F040015961202382F8F7
:101EA4003A30104601F040FA08BD90F83A3010B5C7
:101EB400222B36D183680169B3F5805F0268836A97
:101EC40023D15268E9B9C2F3080223F8022B8362D2
:101ED400C48D013CA4B2C4858CB90368DA6822F0CD
:101EE4002002DA60DA6822F48072DA605A6922F039
:101EF40001025A61202380F83A3001F015FA0020DB
:101F040010BDD2B223F8012BE1E721B9591C526864
:101F140081621A70DCE75268591C816202F07F0208
:101F2400F7E7022010BD704708B5406AFFF7FBFFD2
:101F340008BD7047416A08B50B685A6991F83900C1
:101F440021280AD1120608D50022CA84DA6822F0B0
:101F5400C002DA60202281F839205B6991F83A20C6
:101F6400222A06D15B0604D500230846CB85FFF759
:101F7400D9FDCB6B084643F01003CB63FFF7D9FFC1
:101F840008BD0000036870B51A6804461607D968CE
:101F94005D6907D196065AD58D0658D5BDE87040BF
:101FA400FFF783BF15F0010502D111F4907F4ED0E5
:101FB400D30705D5CE0542BFE36B43F00103E363CA
:101FC400500704D51DB1E36B43F00203E3639307A9
:101FD40004D51DB1E36B43F00403E363160704D592
:101FE4001DB1E36B43F00803E363E36B002B66D09E
:101FF400950604D5880602D52046FFF756FF2368C8
:1020040020465D69E26B110702D415F040051AD031
:10201400FFF788FD23685A69520610D55A69606B28
:1020240022F040025A6150B1254B4363FEF744FA53
:10203400002844D0606BBDE87040436B18472046CD
:10204400FFF777FF70BDFFF774FFE56370BD1606F9
:1020540027D50D0625D594F83920212A2FD1A26839
:10206400B2F5805F226A17D11188C1F30801596063
:10207400216979B902322262E28C013A92B2E28495
:10208400EAB9DA6822F08002DA60DA6842F04002E3
:10209400DA6070BD0132EEE7511C216212785A6099
:1020A400EAE750060BD54A0609D5DA68204622F03D
:1020B4004002DA60202384F83930FFF7D9FE70BD7E
:1020C400C920000808B50023406AC385C384FFF70C
:1020D40030FF08BD70B58178044643185A78013042
:1020E40000F0C9F8C0B201280ED000231E4EA27819
:1020F4005D1C0232DBB29A422EDA1C4801F010FA5F
:1021040022221B4B5A700FE01122194D6A7062781B
:10211400DD2A01D0EE2A07D1204600F0BFFCC0B270
:10212400012801D122236B70114DA978681C00F09D
:1021340087F828716378EE2B06D00A2B04D0A9788F
:102144002846033101F016F96378EE2B0AD1BDE875
:102154007040084801F0E4B9E15C304601F06CF9E4
:102164002B46C4E770BD00BFB0440008B644000865
:1021740008000020C7440008002310B5C11C143017
:1021840011F8014F23448142DBB2F9D19B1A584222
:10219400584110BDC21C00F11403002012F8011FA5
:1021A40008449A42C0B2F9D170470000002310B528
:1021B4000F4CC90007290FDC61B141F2210213F46D
:1021C400004F4FEA43039BB201F1FF3118BF534064
:1021D4000029F4D1184610BD10F8012B083982EA01
:1021E400132234F8122082EA03239BB2E2E700BFF1
:1021F4000E000020002330B5104DC900072911DC62
:1022040061B141F2210013F4004F4FEA43039BB242
:1022140001F1FF3118BF43400029F4D1981A18BFC7
:10222400012030BD10F8014B083984EA132435F835
:10223400144084EA03239BB2E0E700BF0E000020B1
:1022440010B5FF230446221AD2B2914201D818468F
:1022540010BD14F8012B5340082213F0800F02F133
:10226400FF324FEA430318BF83F0310312F0FF0239
:10227400DBB2F2D1E7E730B5FF2305462C1AE4B20E
:10228400A14203D89B1A5842584130BD15F8014B5E
:102294006340082413F0800F04F1FF344FEA430332
:1022A40018BF83F0310314F0FF04DBB2F2D1E5E789
:1022B4004FF0FF3210B5074C0144884201D1D0439E
:1022C40010BD10F8013B5340DBB254F8233083EACD
:1022D4001222F2E7D84400082DE9F04101F120036D
:1022E40023F0070300AFADEB030D04460E46FFF7E2
:1022F4005DFF0DEB0603020A9A750322D8751A7660
:1023040016238DF800308DF801308DF802308DF8E9
:102314000330F12300258DF80530A37968468DF844
:102324000630E3798DF804508DF80730237A8DF860
:1023340011508DF80830637AE8468DF80930A37A95
:102344008DF80A30E37A8DF80B30237B8DF80C304E
:10235400637B8DF80D30A37B8DF80E30E37B8DF815
:102364000F30237C8DF810308DF813508DF81460E5
:10237400FFF710FF2B468DF81500122B1CBF18F821
:102384000320E2540133162BF7D100230133042B2D
:1023940003D12046BD46BDE8F0819A19A1184244F4
:1023A400527D4A75F2E7000010B5837C0446112B78
:1023B40022D003D843B1102B08D010BD132B40D02A
:1023C40032D3142B4AD010BD00F09AFA0323E376DB
:1023D400002323776377A377E37784F8203084F8A6
:1023E40021309023A3740C212046FFF775FFBDE82C
:1023F4001040252100F0BEBFC37E827E1B0403EB88
:102404000263427F1C491344027F03EB02231B4AED
:10241400136000238377C37780F8203080F821305D
:1024240000F068FB9123DDE70323C37600230377E1
:1024340043778377C37780F8203080F82130922364
:10244400D0E70323C3760023037743778377C377E7
:1024540080F8203080F821309323C3E70323C37628
:102464000023037743778377C37780F8203080F89D
:1024740021309423B6E700BF008000089C020020AE
:102484001FB54FF480648DE81C000A4610230146F2
:102494000748FEF751FE0128044605D1054801F01E
:1024A4003FF8204604B010BD1420FDF70DFFF8E7F7
:1024B400D8040020E64A00082DE9F04FC3F347147E
:1024C40087B003F01F0380460F4691460593002C06
:1024D40038D04FF0000A012556461FFA80FBA2456A
:1024E40011DB06F12004A4B2059B43B10026DFF8FA
:1024F40090A0DFF890B02744059B9E4224DB284639
:1025040007B0BDE8F08F4FF48063029320234FEAB5
:102514004A16B6B20193BA1909EB0603009392B2B4
:10252400102359461648FEF771FD0128054605D1CA
:10253400144800F0F5FF0AF1010AD0E71420FDF772
:10254400C3FEF8E70125CFE74FF48063029301232C
:102554000193A3194B44BA19009392B21023414634
:102564005046FEF753FD0128054604D1584600F0B5
:10257400D7FF0136C0E71420FDF7A6FEF9E700BF38
:10258400D8040020E64A00082DE9FF41B94D4FF474
:10259400B0732A464FF42E61A020FFF771FFB648AE
:1025A40000F0BEFFB54B002693F83720B44885F8F9
:1025B400792093F83820B34985F87A2093F83920A4
:1025C40085F87B2093F83A2085F87C2093F83B200B
:1025D40085F87D2093F83C2085F87E20DA7A85F80A
:1025E40076201A7B85F877205B7B85F87830A64BBC
:1025F40093F8372085F8A22093F8382085F8A32093
:1026040093F8392085F8A42093F83A2085F8A5207A
:1026140093F83B2085F8A62093F83C2085F8A72062
:10262400DA7A85F89F201A7B85F8A0205B7B974A8D
:1026340085F8A1300078964B12781B7809780290BF
:10264400944800780190944800780090934800F0F2
:10265400F3FE3146924885F8746000F0EDFE95F87B
:102664007510904800F0E8FE95F87530022B29D1DA
:102674008D4B8E4A1F7801331B781B0443EA076392
:1026840017783B4312F8017C43EA0727884B5C78B0
:102694001A78240444EA0264DA7814439A78854B5D
:1026A40044EA0224621E9A420AD821468248FFF76D
:1026B400FFFDB84200F09180024639467F4829E088
:1026C4003046F6E7012B2CD17D4B7E4A1F7801332F
:1026D4001B781B0443EA076317783B4312F8017C19
:1026E40043EA0727784B5C781A78240444EA0264A6
:1026F400DA7814439A786F4B44EA0224621E9A42B1
:102704000DD821467148FFF7D3FDB84265D039464C
:1027140002466F4804B0BDE8F04100F08DBE30467B
:10272400F3E7032B57D195F87430012B26D1644B72
:102734001A7801331B781B0443EA0263614A127856
:102744001343644A177843EA07275F4B5C781A7887
:10275400240444EA0264DA7814439A78554B44EA30
:102764000224621E9A4207D821465848FFF7A0FD6A
:10277400B842A1D1B8461FE03046F9E737464A4B84
:102784001A7801331B781B0443EA0263474A127820
:102794001343514A92F8008043EA0828444B1C78BA
:1027A40001331B781B0443EA046312F8034C2343EC
:1027B40012F8044C43EA04243E4B621E9A4204D8A5
:1027C40021463D48FFF774FD0746B84505D03A4613
:1027D400414642489EE73446374622462146404811
:1027E40000F02AFE3A4639463E4800F025FE95F8A8
:1027F4007530012B1BD195F87430012B09D03A4860
:1028040000F08EFE39491D4800F0C4F9052385F80F
:1028140075304FF4B073174A4FF42E61A020FFF7C0
:102824004BFE334804B0BDE8F04100F079BE022B02
:102834000CD195F87430022BEBD02E4800F070FECA
:102844002A49114800F0A6F90623E0E703F0FB0348
:10285400032BDED195F87430012B05D1264800F006
:102864005FFE22490848CFE7244800F059FE1F497B
:102874000248E7E728030020D8480008008002083F
:10288400BC7F0008B77F000800800408B87F0008F8
:10289400B97F0008BB7F0008BA7F0008E54800083C
:1028A400134900082B4900084180040844800408A7
:1028B4003D800408FEFF0100808004085B49000895
:1028C40041800208448002083D800208808002089A
:1028D400934900084380020843800408CA49000859
:1028E400024A0008254A00084A4A0008807F000876
:1028F400D04A0008694A0008884A0008AC4A00081F
:102904000C4AB0B5D3690C4C23F01003D3610B4BC4
:102914000B4A1B6800AF0B481360236000F000FEF5
:10292400094B1B6883F308882368BD46BDE8B040A3
:10293400184700BF001002409004002004800008E3
:102944008C0400200C4B0008008000082DE9F041A5
:102954000546044600270F4EDFF83C80AB78621B27
:10296400023B934202DC3846BDE8F0812379E278E9
:10297400316802EB032292B200230120FDF754FFD9
:1029840018B1404600F0CCFD01273368023402330D
:102994003360E3E710020020F14A00082DE9F04714
:1029A400044605464FF00008C37E827E1B0403EBF9
:1029B4000263427F194E1344027FDFF8689003EBF1
:1029C4000223174FDFF860A033603368D9F8002082
:1029D400291B9A1A914205D90133C9F8003040469F
:1029E400BDE8F08795F8233095F82220396802EB8A
:1029F400032292B200230120FDF716FF50B1504686
:102A040000F08EFD4FF47A70FDF75EFC4FF0010884
:102A14000235DAE73B6802333B60F9E7A0020020A5
:102A240088040020E0020020F14A00082DE9F0416A
:102A34000546002690F83E4090F83D30240444EAD0
:102A4400036490F84030134F1C4390F83F30DFF894
:102A5400488044EA03248034A64202D30020BDE81F
:102A6400F081AB195B78AA5D396842EA0322012040
:102A74000023FDF7D9FE40B1404600F051FD4FF46C
:102A84007A70FDF721FC0236E6E73B6802333B60CF
:102A9400F9E700BF88040020F14A000838B5002394
:102AA4000F4C054623600F4BA3604FF6F073E360B1
:102AB400FDF774FE0C4B1A784AB901220B492046E3
:102AC4001A70FDF71BFF10B1094800F029FD2846D4
:102AD400FFF73CFF0446FDF773FE204638BD00BFF8
:102AE400A402002000800008E4020020D402002098
:102AF400FD4A000838B505460C46FDF74FFE194B54
:102B04001A78E2B901211970174B9C42174B1ED059
:102B140017498C4220D0A1F580218C4204D11A603F
:102B2400144A9A603F22DA609A68134B13490F489B
:102B34001A60FDF7E3FE10B1114800F0F1FC2846DD
:102B4400FFF72CFF0446FDF73BFE204638BD1A6014
:102B54000C4A9A600C4AE6E71A600C4A9A600C4ADE
:102B6400E1E700BFE402002000800208B402002074
:102B740000800408807F000888040020D802002018
:102B8400FD4A0008807F0208FFFF1F00807F0408C1
:102B9400BFFF1F002DE9F84307462F480D4600F0FC
:102BA400BFFC3B784A2B04D02C4800F0B9FC01242C
:102BB4004EE00024B8462646DFF8D890414618F87F
:102BC400012B3346FF2A08BF0134484606F10106AB
:102BD40008BFE4B200F030FC802EEFD1642CE6D8BC
:102BE4001D4800F09DFCFDF7D9FD1D4B1C781CBB56
:102BF40001221C481A7000F093FC1B4B9D420AD121
:102C040029461A4800F018FC4022194B1C609D60AC
:102C1400DA60184B1D60184800F082FC174800F079
:102C24007FFC17491248FDF769FE10B1154800F002
:102C340077FC154800F074FC144800F071FC384629
:102C4400FFF7F4FE0446124800F06AFCFDF7B8FDF5
:102C54002046BDE8F88300BF124B0008424B000831
:102C6400E4020020684B0008807F00088E4B0008B7
:102C7400C402002088040020A24B0008C64B0008B0
:102C8400DC020020FD4A0008DD4B0008F24B00087E
:102C9400044C00084E4B00080268084B9A420BD1C2
:102CA400074A136801331360064A1368013313603B
:102CB400054A136801331360704700BF00100040D9
:102CC400F0020020EC020020E802002010B51446B7
:102CD4000A230248FFF728F8204610BD7806002092
:102CE40010B590B02822002106A800F09DFB142204
:102CF400002101A800F098FB01230A931023022469
:102D04000B934FF4401306A80F9306940D94FEF70B
:102D140033FB0F234FF4806201930023214601A863
:102D24000294039304920593FEF7EEFC10B010BDD9
:102D340080B588B0FDF7A4FAFFF7D2FF1022644DE6
:102D440000210DEB020000F06FFBAB69002243F0A1
:102D54001003AB61AB694FF4004103F0100301931E
:102D6400019BAB695B4843F00403AB61AB6900248E
:102D740003F004030293029BAB694FF4E13743F081
:102D84000803AB61AB690C2603F008030393039BB0
:102D9400FDF7EEFE4FF40043049301230593022351
:102DA40004A94C4807930694FDF7F6FD6B694A485D
:102DB40043F001036B616B69846003F001030093CA
:102DC400009B464BC46080E88800046146618461CE
:102DD400C461FEF77BFF4248424A434B846080E86B
:102DE4000C004FF48043C460036144618461C46196
:102DF4000462FEF78BF841F2DF533C4D3C49284610
:102E040085E80A0009230494EB600594AC60AC6186
:102E1400FEF74AFE04A9284604940594FEF75EFED4
:102E2400344B354880E888008460C460046146619E
:102E34008461C461FEF74AFF224621460F20FDF754
:102E440067FA0F20FDF798FA224621462520FDF760
:102E54005FFA2520FDF790FA224621463620FDF739
:102E640057FA3620FDF788FA224621460E20FDF750
:102E74004FFA0E20FDF780FA224621462620FDF760
:102E840047FA2620FDF778FA224621461020FDF75E
:102E94003FFA1020FDF770FA224621461120FDF773
:102EA40037FA1120FDF768FA2846FEF7FFFC134BAA
:102EB40021461B68986800F03BFB114800F030FB8A
:102EC400FFF762FB0F4800F02BFBFFF719FDFEE74D
:102ED4000010024000100140F805002000380140B5
:102EE400D804002000580040801A0600380600204C
:102EF4000010004000440040780600201802002022
:102F0400144C0008234C0008704700000E4B82B09C
:102F14009A6942F001029A619A6902F001020092F0
:102F2400009ADA6942F08052DA61DB69074A03F0F9
:102F340080530193019B536823F0E06343F00073D3
:102F4400536002B0704700BF00100240000001400F
:102F540010B5044686B01022002102A800F064FADD
:102F64002268114B9A421DD1104C02A9A369104842
:102F740043F00803A361A36903F008030093009BD3
:102F84004FF4406302931223039303230593FDF745
:102F940003FDE36943F48003E361E36903F480031D
:102FA4000193019B06B010BD005800400010024080
:102FB400000C01400268084B82B09A420AD103F522
:102FC4000033DA6942F01002DA61DB6903F01003BE
:102FD4000193019B02B0704700100040102270B5AD
:102FE400054688B00DEB0200002100F01DFA2B68A5
:102FF400494A934251D1494B04A99A69484842F439
:1030040080429A619A69002602F480420092009AF2
:103014009A69444C42F004029A619B6903F00403E8
:103024000193019B4FF4007304930223059303233C
:103034000793FDF7B1FC4FF48063394804A9049366
:1030440005960696FDF7A8FC374B204684E8480011
:103054008023A660E36026616661A661E661FDF7F0
:10306400ADF908B1FFF750FF6C6365622F4B304C2C
:1030740023601023802263600023E260A360236145
:103084006361A361E3612046FDF798F908B1FFF796
:103094003BFF2C63656208B070BD264A9342FAD1A7
:1030A4001E4B04A9DA691E4842F40032DA61DA6977
:1030B400002602F400320292029A9A691E4C42F0EF
:1030C40004029A619B6903F004030393039B0423A2
:1030D40004930223059303230793FDF75DFC082360
:1030E4000F4804A9049305960696FDF755FC134B67
:1030F400204684E848008023A660E3602661666178
:10310400A661E661FDF75AF908B1FFF7FDFE6C63AD
:1031140065620B4B0B4CABE70038014000100240DA
:10312400000801407005002058000240440002409D
:103134002C05002000440040940400206C00024050
:1031440080000240B40500207047FEE7FEE7FEE77A
:10315400FEE7704770477047FDF7A4B80148FDF7D4
:1031640019BA00BF2C0500200148FDF713BA00BFAF
:10317400700500200148FDF70DBA00BF940400203B
:103184000148FDF707BA00BFB40500200148FEF767
:10319400F9BE00BFF80500200148FEF7F3BE00BFEA
:1031A400780600200148FEF790BB00BF38060020D7
:1031B40070B50E4615460C46A31B9D4201DC2846FD
:1031C40070BDAFF3008004F8010BF5E708B50A4BB6
:1031D4000246196809B90949196069461868024420
:1031E4008A4206D900F0F6F80C2303604FF0FF3052
:1031F40008BD1A6008BD00BFF4020020B813002007
:103204004FF0FF3070474FF4005300204B6070477D
:1032140001207047002070470F4B1A6842F00102EA
:103224001A6059680D4A0A405A601A6822F084727A
:1032340022F480321A601A6822F480221A605A68D2
:1032440022F4FE025A604FF41F029A604FF00062AB
:10325400034B9A60704700BF001002400000FFF863
:1032640000ED00E0294A70B51068294C431C136036
:10327400284B596803F10C054D5D0131255440F28A
:103284004B408142C8BF00219D685960013D9D604B
:103294007DB923781560BE2B0CD11D48FEF71AFFAB
:1032A400002340F24C42635501359542FBD11A4A42
:1032B400136070BD162BF3D16378162BF0D1A3786D
:1032C400162BEDD1E378162BEAD1627D122110483A
:1032D400FEF752FFB0B1E37C217D104841EA03219F
:1032E4006318DA7D1E7E46EA02263246FEF782FF26
:1032F40018B10748FFF758F8D2E73146084800F0FC
:103304009BF8CDE7617D0748F9E700BFF80200208C
:10331400100B0020B8060020E8020020260B002035
:10332400454C0008534C000800220E4B10B51A609F
:1033340040F24B420C4C236801339342C8BF002334
:103344002360A36801339342A36001DDFFF78AFF82
:10335400236806490122BDE8104019440448FEF7D9
:103364003FBD00BFF0020020B8060020C4060020C4
:10337400F80500200A464FF6FF7301460148FEF7A0
:10338400D3BC00BFF8050020002103E00B4B5B58C1
:10339400435004310A480B4B42189A42F6D30A4A66
:1033A40002E0002342F8043B084B9A42F9D3FFF7AA
:1033B40033FF00F015F8FFF7BBFC7047084D000819
:1033C400000000207C02002080020020B8130020AE
:1033D400FEE70000014B1868704700BF1802002088
:1033E40070B500250C4E0D4CA41BA410A54209D1A8
:1033F40001F048F800250A4E0A4CA41BA410A5426B
:1034040005D170BD56F8253098470135EEE756F8DA
:10341400253098470135F2E7004D0008004D0008BB
:10342400004D0008044D000803460244934200D1B5
:10343400704703F8011BF9E70FB40A4B13B51C6876
:1034440024B1A36913B9204600F0DAFA05AB049A53
:10345400A1682046019300F09BFC02B0BDE8104037
:1034640004B070471802002070B50E46054618B126
:1034740083690BB900F0C4FAAB69AC6813B9284688
:1034840000F0BEFA234B9C4217D16C68A3891B073A
:103494001DD52369DBB1013EA36816F8011F013B6A
:1034A400A360E9B9002B2EDA22460A21284600F04F
:1034B400F5F8013011D00A2070BD174B9C4201D1A0
:1034C400AC68E3E7154B9C4208BFEC68DEE7214695
:1034D400284600F035F90028DDD04FF0FF3070BDEC
:1034E400002B04DAA269934206DB0A2904D023687C
:1034F4005A1C22601970CFE72246284600F0CEF805
:103504000130C9D1E9E70A2023685A1C22601870E7
:1035140070BD00BF8C4C0008AC4C00086C4C00081B
:10352400024B01461868FFF79FBF00BF1802002036
:1035340000294FF480630CBF0222002200F000B87F
:103544002DE9F7431D46514B04461E680F4690462D
:1035540026B1B36913B9304600F052FA4C4B9C4281
:1035640052D17468B8F1020F06D0B8F1010F00F21D
:103574008980002DC0F286802146304600F0D6F9BD
:10358400616B41B104F14403994202D0304600F02A
:103594002DFB002363630023A3616360A3891B06DF
:1035A40003D52169304600F021FBA389B8F1020F4D
:1035B40023F44A6323F00303A3815DD001AB6A467D
:1035C4002146304600F0A6FAA3891843A0812DBBFA
:1035D400009D284600F002FB074600284ED1DDF886
:1035E4000090A9453CD14FF0FF30A38943F002037A
:1035F400A3810023A36004F1470323602361012313
:10360400636103B0BDE8F083224B9C4201D1B468EE
:10361400A8E7214B9C4208BFF468A3E7002FD8D049
:10362400B36913B9304600F0EBF9B8F1010F08BFE4
:10363400A389276004BF43F00103A381A389276101
:1036440013F0080065611BD013F001004FF0000374
:103654001FBF6D42A360A561184608BFA560D0E7EF
:10366400484600F0BBFA07460028BCD0A3894D4663
:1036740043F08003A381D3E70020B6E7A946F5E72A
:10368400A060BEE74FF0FF30BBE700BF1802002088
:103694008C4C0008AC4C00086C4C0008F8B50E4685
:1036A4001446054618B183690BB900F0A9F9214BFA
:1036B4009C422AD16C68A369A360A3891A072ED5FA
:1036C400236963B323692068F6B2C01A6369374675
:1036D400984204DB2146284600F028F928BBA36859
:1036E4000130013BA36023685A1C22601E70636989
:1036F400984204D0A389DB0719D50A2E17D1214695
:10370400284600F013F990B10FE00B4B9C4201D115
:10371400AC68D0E7094B9C4208BFEC68CBE7214674
:10372400284600F00DF80028CCD04FF0FF3738467B
:10373400F8BD00BF8C4C0008AC4C00086C4C000871
:10374400324B70B51D6806460C4625B1AB6913B9FA
:10375400284600F055F92E4B9C420FD16C68B4F901
:103764000C309AB215072CD4D00611D40922326039
:1037740043F04003A3814FF0FF3070BD254B9C42C2
:1037840001D1AC68EBE7244B9C4208BFEC68E6E748
:10379400510712D5616B41B104F14403994202D03F
:1037A400304600F023FA00236363A38923F0240343
:1037B400A3810023636023692360A38943F0080382
:1037C400A38123694BB9A38903F42073B3F5007F64
:1037D40003D02146304600F0C1F9A28912F001035A
:1037E4000CD00023A36063695B42A361236953B9CE
:1037F400B4F90C3013F08000BAD170BD920758BFF1
:103804006369A360F2E70020F7E700BF1802002015
:103814008C4C0008AC4C00086C4C00088A892DE9DB
:10382400F041054610070C465AD44B68002B05DCC2
:103834000B6C002B02DC0020BDE8F081E66A002E50
:10384400F9D0002312F480522F682B6033D0606DBE
:10385400A3895A0705D56368C01A636B0BB1236C3F
:10386400C01A00230246E66A216A2846B047431C70
:10387400A38906D129681D294BD82B4ACA40D607EB
:1038840047D5002262602269D904226004D5421C13
:1038940001D12B6803B96065616B2F600029CAD020
:1038A40004F14403994202D0284600F09FF9002015
:1038B4006063BDE8F081216A01232846B047411CBA
:1038C400C6D12B68002BC3D01D2B01D0162B01D1E0
:1038D4002F60B0E7A38943F04003A381BDE8F081E2
:1038E4000F69002FA7D0930718BF00230E6808BFE5
:1038F4004B69A6EB07080F608B60B8F1000F9ADDE7
:1039040043463A46216A2846A66AB047002807DC9F
:10391400A38943F04003A3814FF0FF30BDE8F08159
:103924000744A8EB0008E8E70100402038B50B691C
:1039340005460C46DBB118B183690BB900F060F899
:103944000C4B9C4209D16C68B4F90C307BB1214614
:103954002846BDE83840FFF761BF074B9C4201D1C0
:10396400AC68F1E7054B9C4208BFEC68ECE700202B
:1039740038BD00BF8C4C0008AC4C00086C4C0008EF
:10398400014900F0A9B800BF31390008002310B57F
:10399400044603604360836081814366C28103619E
:1039A40043618361194608225C30FFF73DFD054BF6
:1039B40024626362044BA362044BE362044B2363FB
:1039C40010BD00BF11430008334300086B430008D7
:1039D4008F43000870B568254A1E55430E4605F10D
:1039E400740100F04FF9044640B1002180E8420020
:1039F4000C30A06005F16802FFF716FD204670BD8B
:103A0400836910B5044633BB8364C3640365124BF6
:103A1400124A1B688262984204BF0123836100F04A
:103A24001FF86060204600F01BF8A060204600F0FC
:103A340017F80022E06004216068FFF7A7FF012265
:103A44000921A068FFF7A2FF02221221E068FFF714
:103A54009DFF0123A36110BD684C0008853900084F
:103A6400F8B51C4B07461E68B36913B93046FFF717
:103A7400C7FF4836B4687368013B03D5336833B174
:103A84003668F7E7B4F90C506DB16834F4E70421F3
:103A94003846FFF79FFF30600028F1D10C2304461D
:103AA4003B602046F8BD4FF6FF73E3810123656652
:103AB400A3812560A560656025616561A561082213
:103AC400294604F15C00FFF7AFFC6563A563A564B8
:103AD400E564E6E7684C00082DE9F843804689462A
:103AE400002600F1480414B93046BDE8F883A568FF
:103AF4006768013F01D52468F5E7AB89012B07D935
:103B0400B5F90E30013303D029464046C847064371
:103B14006835EEE770B50E46B1F90E1090B0002985
:103B240014461D4607DA00232B60B3891A0610D405
:103B34004FF480630EE001AA00F04EFC0028F2DB93
:103B4400029A02F47042A2F500535A425A412A6082
:103B5400EEE740230020236010B070BD8B8973B55D
:103B64009D0706460C4607D504F1470323602361ED
:103B74000123636102B070BD01AB6A46FFF7CAFF5F
:103B840000990546304600F07DF848B9B4F90C3088
:103B94009A05EFD423F0030343F00203A381E3E780
:103BA4000D4BB362A389206043F08003A381009B83
:103BB40020616361019B5BB1B4F90E10304600F0E3
:103BC4001DFC28B1A38923F0030343F00103A3815F
:103BD400A3891D43A581CDE785390008024B014621
:103BE400186800F04FB800BF1802002038B5054629
:103BF400002943D051F8043C0C1F002BB8BFE41833
:103C040000F02CFC1E4A1368104633B9636014603C
:103C14002846BDE8384000F022BCA3420BD92168F5
:103C24006218934201BF1A685B685218226063608D
:103C34000460EDE713465A680AB1A242FAD919683A
:103C44005818A0420BD120680144581882421960C8
:103C5400DED110685268014419605A60D8E702D96D
:103C64000C232B60D4E7206821188A4201BF116815
:103C740052680918216062605C60C9E738BD00BF02
:103C8400FC02002070B5CD1C25F0030508350C2D71
:103C940038BF0C25002D064601DBA94203D90C23AD
:103CA4003360002070BD00F0D9FB234A146821461C
:103CB40091B9224C23681BB9304600F017FB2060F1
:103CC4002946304600F012FB431C26D10C23304613
:103CD400336000F0C4FBE4E70B685B1B1AD40B2BC6
:103CE4000FD90B60CC18CD50304600F0B8FB04F16E
:103CF4000B00231D20F00700C31A1BD05A42E250C8
:103D040070BD8C420BBF63684B681360636018BF5F
:103D14000C46E9E70C464968CAE7C41C24F00304CE
:103D2400A04205D0211A304600F0E0FA0130CDD08F
:103D34002560D9E770BD00BFFC020020000300200D
:103D4400936810B4013B002B936008DA9469A34292
:103D540002DBCBB20A2B02D110BCFFF79FBC136865
:103D6400581C10601970C8B210BC7047F8B50646EC
:103D74000F461446D518AC4201D1002007E03A465C
:103D840014F8011B3046FFF7DBFF431CF3D1F8BDE9
:103D94002DE9F04F9DB00C4617460393064618B123
:103DA40083690BB9FFF72CFE7C4B9C4257D1746896
:103DB400A38918075DD52369002B5AD000230993E2
:103DC40020238DF8293030234FF0010B8DF82A3051
:103DD400B846454615F8013B002B55D1B8EB070A08
:103DE4000BD053463A4621463046FFF7BFFF013019
:103DF40000F0C480099B5344099398F80030002BC9
:103E040000F0BC8000234FF0FF3204930793059227
:103E140006938DF853301A9305222978604800F0F0
:103E24000FFB05F10108049B002831D1D90644BFDA
:103E340020228DF853201A0744BF2B228DF85320DB
:103E44002A782A2A2CD000210A20079AA84698F812
:103E540000300135303B092B6DD971B326E0514B4D
:103E64009C4201D1B468A3E74F4B9C4208BFF4685D
:103E74009EE721463046FFF763FC00289ED04FF0B2
:103E8400FF301DB0BDE8F08F252BA7D0A846A0E7D2
:103E9400434A4546801A0BFA00F018430490BBE7E6
:103EA400039A111D12680391002A01DB079204E0B2
:103EB400524243F002030792049398F800302E2BE9
:103EC40010D198F8013008F101012A2B37D1039B56
:103ED40008F102081A1D1B680392002BB8BF4FF0AB
:103EE400FF330593314D032298F80010284600F063
:103EF400A7FA40B14023401B03FA00F0049B08F1E9
:103F040001080343049398F800100622284808F196
:103F140001078DF8281000F093FA002834D0254BBF
:103F240003BB039B073323F0070308330393099B65
:103F34004B4409934CE700FB0232012186E700233E
:103F44000A2518460593884698F800200131303A2E
:103F5400092A03D9002BC5D00590C3E705FB00202F
:103F64000123F0E703AB00932246134B04A9304628
:103F7400AFF30080B0F1FF3F8146D8D1A3895B063F
:103F84003FF57DAF09987CE703AB009322460A4BCB
:103F940004A9304600F08AF8ECE700BF8C4C000816
:103FA400CC4C0008AC4C00086C4C0008D24C000807
:103FB400D64C000800000000713D00082DE9F047D0
:103FC40091461F468A680B6906469342B8BF13465A
:103FD400C9F8003091F843200C46DDF8208012B176
:103FE4000133C9F800302368990642BFD9F800307C
:103FF4000233C9F80030256815F0060507D104F12D
:10400400190AE368D9F800209B1A9D422ADB94F828
:1040140043302268003318BF012392062FD404F1E1
:10402400430239463046C047013022D02368E56850
:1040340003F00603042B18BF0025D9F800204FF025
:10404400000908BFAD1AA368226908BF25EAE5750F
:104054009342C4BF9B1AED181A344D451BD100205E
:10406400BDE8F0870123524639463046C047013047
:1040740003D14FF0FF30BDE8F0870135C1E73020B0
:10408400E11881F843005A1C94F845102244023385
:1040940082F84310C3E70123224639463046C0471D
:1040A4000130E6D009F10109D7E700002DE9F0431A
:1040B40017460A7E85B06E2A984606460C460C9B27
:1040C40001F1430E00F0BC801AD8632A2ED00AD81E
:1040D400002A00F0C880582A00F08A8004F14205C2
:1040E40084F842202AE0642A01D0692AF6D12168A2
:1040F4001A6811F0800F23D0111D1960136827E08E
:10410400732A00F0B48008D86F2A2AD0702AE5D127
:104114000A6842F020020A6003E0752A21D0782A56
:10412400DCD178226F4984F8452064E01A6801F1F3
:104134004205111D1960136884F842300123A3E07D
:1041440011F0400F02F104011960D7D0B2F9003028
:10415400002B03DA2D225B4284F8432062490A22B1
:1041640017E02068196810F0800F03D0081D18604C
:104174000B6806E010F0400F01F104001860F7D05E
:104184000B886F2A14BF0A2208225749002084F89A
:1041940043006568002DA560C0F29C80206820F073
:1041A40004002060002B3FD1002D40F0958075461F
:1041B400082A0BD12368DA0708D5236962689A4272
:1041C400DEBF302305F8013C05F1FF35AEEB0503F6
:1041D4002361CDF800803B4603AA21463046FFF711
:1041E400EDFE013055D14FF0FF3005B0BDE8F0834E
:1041F40081F845203C492268186812F0800F00F1CC
:1042040004051D6001D0036802E05506FBD5038850
:10421400D00744BF42F0200222601BB9226822F07A
:10422400200222601022B1E77546B3FBF2F002FBD4
:104234001033CB5C05F8013D03460028F5D1B7E700
:1042440008681A6810F0800F496904D0101D1860BE
:104254001368196007E010F0400F02F104001860C1
:104264001368F6D01980002375462361B1E71A68F4
:10427400111D1960156800216268284600F0E0F8F5
:1042840008B1401B606063682361002384F84330F5
:104294009FE723692A4639463046C0470130A2D0F9
:1042A40023689B0707D5002504F11909E368039ADD
:1042B4009B1A9D4205DBE068039B9842B8BF1846F1
:1042C40093E701234A4639463046C04701308AD035
:1042D4000135EBE7002BA7D10B7804F1420584F8F4
:1042E400423065E7EE4C0008DD4C000838B5002389
:1042F400054C054608462360FEF768FF431C02D1BF
:10430400236803B12B6038BDB413002010B50C46EC
:10431400B1F90E1000F0A4F80028ABBF636DA389B7
:104324001B1823F48053ACBF6365A38110BD2DE932
:10433400F0411F468B890546DB050C46164605D51C
:1043440002230022B1F90E1000F068F8A389324666
:1043540023F48053A381B4F90E103B462846BDE8EC
:10436400F04100F017B810B50C46B1F90E1000F08A
:1043740055F8431CA38915BF606523F4805343F4A7
:104384008053A38118BFA38110BDB1F90E1000F0B2
:1043940013B8000038B50546084611460022054CFE
:1043A40022601A46FEF792FC431C02D1236803B133
:1043B4002B6038BDB413002038B50023054C0546E6
:1043C40008462360FEF71CFF431C02D1236803B197
:1043D4002B6038BDB413002038B50023064C0546C5
:1043E400084611462360FEF70EFF431C02D12368E2
:1043F40003B12B6038BD00BFB413002038B50023CF
:10440400054C054608462360FEF702FF431C02D113
:10441400236803B12B6038BDB413002038B50546BA
:10442400084611460022054C22601A46FEF7F2FEA9
:10443400431C02D1236803B12B6038BDB4130020A0
:1044440010B5C9B202449042034601D1002010BD08
:104454001C7801308C42F6D1184610BD7047704765
:1044640038B50546084611460022054C22601A4616
:10447400FEF79EFE431C02D1236803B12B6038BDB6
:10448400B4130020F8B500BFF8BC08BC9E467047C2
:0C449400F8B500BFF8BC08BC9E4670479D
:1044A00002030405060708090A0B0C0D0E0F101075
:1044B000253032782000436865636B2053756D208A
:1044C0006572726F72200075706461746520436F4D
:1044D0006D706C65746520000000000096300777F1
:1044E0002C610EEEBA51099919C46D078FF46A70E8
:1044F00035A563E9A395649E3288DB0EA4B8DC7908
:104500001EE9D5E088D9D2972B4CB609BD7CB17E87
:10451000072DB8E7911DBF906410B71DF220B06A57
:104520004871B9F3DE41BE847DD4DA1AEBE4DD6D67
:1045300051B5D4F4C785D38356986C13C0A86B6467
:104540007AF962FDECC9658A4F5C0114D96C066387
:10455000633D0FFAF50D088DC8206E3B5E10694C67
:10456000E44160D5727167A2D1E4033C47D4044BA7
:10457000FD850DD26BB50AA5FAA8B5356C98B24287
:10458000D6C9BBDB40F9BCACE36CD832755CDF4507
:10459000CF0DD6DC593DD1ABAC30D9263A00DE5137
:1045A0008051D7C81661D0BFB5F4B42123C4B35627
:1045B0009995BACF0FA5BDB89EB802280888055FA7
:1045C000B2D90CC624E90BB1877C6F2F114C685807
:1045D000AB1D61C13D2D66B69041DC760671DB01F5
:1045E000BC20D2982A10D5EF8985B1711FB5B606C7
:1045F000A5E4BF9F33D4B8E8A2C9077834F9000F07
:104600008EA8099618980EE1BB0D6A7F2D3D6D08A6
:10461000976C6491015C63E6F4516B6B62616C1C96
:10462000D83065854E0062F2ED95066C7BA5011BC6
:10463000C1F4088257C40FF5C6D9B06550E9B71266
:10464000EAB8BE8B7C88B9FCDF1DDD62492DDA1526
:10465000F37CD38C654CD4FB5861B24DCE51B53A46
:104660007400BCA3E230BBD441A5DF4AD795D83D46
:104670006DC4D1A4FBF4D6D36AE96943FCD96E3486
:10468000468867ADD0B860DA732D0444E51D033366
:104690005F4C0AAAC97C0DDD3C710550AA41022776
:1046A00010100BBE86200CC925B56857B3856F2046
:1046B00009D466B99FE461CE0EF9DE5E98C9D929A6
:1046C0002298D0B0B4A8D7C7173DB359810DB42EE6
:1046D0003B5CBDB7AD6CBAC02083B8EDB6B3BF9A32
:1046E0000CE2B6039AD2B1743947D5EAAF77D29DBE
:1046F0001526DB048316DC73120B63E3843B64949E
:104700003E6A6D0DA85A6A7A0BCF0EE49DFF09939D
:1047100027AE000AB19E077D44930FF0D2A308870D
:1047200068F2011EFEC206695D5762F7CB676580BD
:1047300071366C19E7066B6E761BD4FEE02BD389BD
:104740005A7ADA10CC4ADD676FDFB9F9F9EFBE8E1D
:1047500043BEB717D58EB060E8A3D6D67E93D1A15D
:10476000C4C2D83852F2DF4FF167BBD16757BCA63D
:10477000DD06B53F4B36B248DA2B0DD84C1B0AAFDD
:10478000F64A0336607A0441C3EF60DF55DF67A85D
:10479000EF8E6E3179BE69468CB361CB1A8366BCED
:1047A000A0D26F2536E2685295770CCC03470BBB3D
:1047B000B91602222F260555BE3BBAC5280BBDB23D
:1047C000925AB42B046AB35CA7FFD7C231CFD0B5DD
:1047D0008B9ED92C1DAEDE5BB0C2649B26F263ECCF
:1047E0009CA36A750A936D02A906099C3F360EEBDD
:1047F0008567077213570005824ABF95147AB8E29D
:10480000AE2BB17B381BB60C9B8ED2920DBED5E57C
:10481000B7EFDC7C21DFDB0BD4D2D38642E2D4F1CC
:10482000F8B3DD686E83DA1FCD16BE815B26B9F65C
:10483000E177B06F7747B718E65A0888706A0FFFBC
:10484000CA3B06665C0B0111FF9E658F69AE62F87C
:10485000D3FF6B6145CF6C1678E20AA0EED20DD77C
:104860005483044EC2B30339612667A7F71660D09C
:104870004D476949DB776E3E4A6AD1AEDC5AD6D9DC
:10488000660BDF40F03BD83753AEBCA9C59EBBDEFC
:104890007FCFB247E9FFB5301CF2BDBD8AC2BACAAC
:1048A0003093B353A6A3B4240536D0BA9306D7CD1C
:1048B0002957DE54BF67D9232E7A66B3B84A61C43C
:1048C000021B685D942B6F2A37BE0BB4A18E0CC3FC
:1048D0001BDF055A8DEF022D466C61736820496E0F
:1048E0006974200D00323025642059202F20256462
:1048F000204D202F2025642044202F20256420488F
:10490000202F202564204D202F2025642053202097
:104910000D0A004D4249432042414E4B2025642060
:10492000426F6F74696E67200D0A00626C75656373
:10493000656C6C5F437572726461746173746174E9
:1049400075732E4350555F42616E6B5F53656C65A6
:104950006374203A202564200D0A0042616E6B3199
:104960002043524320455252203A2046494C45208C
:10497000435243203A20257820202F2F2F2020201B
:104980002043414C432020435243203A20257820A5
:104990000D0A0042616E322043524320455252209C
:1049A0003A2046494C4520435243203A202578205E
:1049B000202F2F2F2020202043414C4320204352E2
:1049C00043203A202578200D0A0042616E6B322088
:1049D00043524320455252203A2046494C452043F9
:1049E0005243203A20257820202F2F2F20202020CE
:1049F00043414C432020435243203A202578200D48
:104A00000A00435243204C454E475448203A202543
:104A1000642C435243204C454E475448203A2025AD
:104A200058200D0A004352432053554343455353E6
:104A300020203A202578202C2046696C652043529E
:104A400043203A202578200D0A00577269746520AA
:104A500053746172742042414E4B203120446F7771
:104A60006E2053746172740D00577269746520531F
:104A7000746172742042414E4B203220446F776E35
:104A80002053746172740D005772697465205374F9
:104A90006172742042414E4B2042414E4B203120E6
:104AA000446F776E2053746172740D00577269748D
:104AB000652053746172742042414E4B2042414E36
:104AC0004B203220446F776E2053746172740D0056
:104AD000454550524F4D20494E495420434F4D506B
:104AE0004C4554450D005772697465204552520D6E
:104AF0000048414C204E4F54204F4B2000457261DE
:104B00007365204661696C6564200D006A756D707F
:104B100021003D3D3D3D3D3D3D3D3D3D3D3D3D3D1E
:104B20003D3D3D3D3D3D3D446174612052656376B0
:104B30003D3D3D3D3D3D3D3D3D3D3D3D3D3D3D3DA5
:104B40000D0046696C65204552526F720D0025308C
:104B50003878203A20253032582020496E64657814
:104B6000203A202564200A00446F776E6C6F6164E0
:104B700020457261736520436F6E69666967756170
:104B8000726174696F6E2053746172740D00557395
:104B90006572204150492045726173652025780D6A
:104BA0000A00446F776E6C6F6164204572617365B3
:104BB00020436F6E696669677561726174696F6EB3
:104BC00020454E440D00446F776E6C6F6164204544
:104BD00072617365202073746172740D00446F7785
:104BE0006E6C6F61642045726173652020454E4490
:104BF0000D00446F776E6C6F616420537461727442
:104C000020200D00446F776E6C6F616420454E4428
:104C100020200D00426F6F745374617274202D2D2B
:104C20002D0D00426F6F7420454E440D00000000B2
:104C3000000000000001020304060708090000004C
:104C4000000102030443524320455252202578209C
:104C50000D0A00434845434B2053554D20455252C1
:104C6000202578200D0A00001C0200200000000012
:104C70000000000000000000000000000000000034
:104C80000000000000000000000000000000000024
:104C90000000000000000000000000000000000014
:104CA0000000000000000000000000000000000004
:104CB00000000000000000000000000000000000F4
:104CC000000000000000000000000000232D302B39
:104CD0002000686C4C0065666745464700303132FD
:104CE0003334353637383941424344454600303154
:104CF00032333435363738396162636465660000B3
:044D0000090200089C
:044D0400E5010008BD
:104D08000100000010000000BE11030500BE0000F5
:104D18002110422063308440A550C660E7700881A6
:104D280029914AA16BB18CC1ADD1CEE1EFF131121D
:104D3800100273325222B5529442F772D6623993F6
:104D480018837BB35AA3BDD39CC3FFF3DEE362246D
:104D5800433420040114E664C774A44485546AA546
:104D68004BB528850995EEE5CFF5ACC58DD55336FD
:104D7800722611163006D776F6669556B4465BB796
:104D88007AA719973887DFF7FEE79DD7BCC7C448CD
:104D9800E5588668A7784008611802282338CCC9E6
:104DA800EDD98EE9AFF9488969990AA92BB9F55A5D
:104DB800D44AB77A966A711A500A333A122AFDDB36
:104DC800DCCBBFFB9EEB799B588B3BBB1AABA66C2D
:104DD800877CE44CC55C222C033C600C411CAEED86
:104DE8008FFDECCDCDDD2AAD0BBD688D499D977E3D
:104DF800B66ED55EF44E133E322E511E700E9FFFD6
:104E0800BEEFDDDFFCCF1BBF3AAF599F788F88918B
:104E1800A981CAB1EBA10CD12DC14EF16FE180106F
:104E2800A100C230E3200450254046706760B98372
:104E38009893FBA3DAB33DC31CD37FE35EF3B102BF
:104E48009012F322D2323542145277625672EAB582
:104E5800CBA5A89589856EF54FE52CD50DC5E2340F
:104E6800C324A01481046674476424540544DBA752
:104E7800FAB79987B8975FE77EF71DC73CD7D3265F
:104E8800F2369106B01657667676154634564CD9E2
:104E98006DC90EF92FE9C899E9898AB9ABA94458AF
:104EA800654806782768C018E1088238A3287DCBB2
:104EB8005CDB3FEB1EFBF98BD89BBBAB9ABB754AFF
:104EC800545A376A167AF10AD01AB32A923A2EFD42
:104ED8000FED6CDD4DCDAABD8BADE89DC98D267C4F
:104EE800076C645C454CA23C832CE01CC10C1FEF92
:104EF8003EFF5DCF7CDF9BAFBABFD98FF89F176E9F
:104F0800367E554E745E932EB23ED10EF01E0000D2
:104F18000080000800A24A041C02002000000000D3
:104F28008C4C0008AC4C00086C4C000800000000D9
:104F38000000000000000000000000000000000069
:104F48000000000000000000000000000000000059
:104F58000000000000000000000000000000000049
:104F68000000000000000000000000000000000039
:0C4F78000000000000000000000000002D
:040000050800338D2F
:00000001FF
